:100000003BC072C153C052C051C050C04FC04EC05F
:100010004DC04CC04BC04AC049C048C047C046C094
:1000200045C044C043C00E03550053004200610068
:10003000730070001C037700770077002E006600C5
:1000400069007300630068006C002E0064006500A6
:1000500004030904090212000101008019090400C7
:1000600000000000000012010101FF000008EB0386
:10007000B4C700010102000111241FBECFE5D4E086
:10008000DEBFCDBF10E0A0E6B0E0EAEAFCE002C0CF
:1000900005900D92A436B107D9F710E0A4E6B0E0C0
:1000A00001C01D92A23AB107E1F7EAC5A9CF1F939B
:1000B000CF93FC0180919B008D3269F080917A0092
:1000C00087FD04C0CF014DD58F3F71F010926300C2
:1000D00010927A0066C0C0E010E8683061F0C0930A
:1000E000630010937A005DC08EE180938D0082E002
:1000F0008093620056C080818076F9F426E930E072
:10010000C093960081818823A1F08530E9F0863084
:10011000F9F0883061F18A3071F130939D002093BD
:100120009C0087818823D9F686818C17C0F6C82F5A
:10013000D6CFC0939700C2E0F0CFC681CF0104D4E0
:100140008F3FA9F710E0CBCF828180937B00E5CF72
:1001500010EC8381813089F0823099F08330E9F6A8
:100160008281882391F4C4E020E530E0D6CFC1E05D
:10017000C0939600D2CFC1E0D0CFC2E126E630E0F6
:10018000CCCFC2E124E530E0C8CF813031F08230FD
:1001900021F6CEE026E230E0C0CFCCE124E330E02F
:1001A000BCCFCF911F910895CF9360919E0066239D
:1001B00051F0635067FD05C0809199009927019621
:1001C00076DF10929E008091620087FD1AC086B390
:1001D000837019F010927C0077C080917C00882396
:1001E00009F072C094E686B3837009F06DC0915037
:1001F000D1F781E080937C009093980090937B00EE
:1002000063C0809163008F3F31F12BE490917A00BD
:1002100090FD23EC9F5F90937A0020938D00682FD0
:10022000893008F068E0861B80936300AEE8B0E098
:1002300097FD30C0662349F560E070E0C62F693055
:10024000A0F08EE180938D0092E08FEF80936300A9
:1002500090936200BCCF80917B00882309F4B7CFD4
:100260008093980010927B00B2CF8EE890E0C1D1CD
:10027000EC2FFF27E357FF4F818392839C2F9C5FD6
:10028000C83018F390936200A2CFCD012DD4682F0F
:100290007727D4CFE0919C00F0919D0096FF0DC090
:1002A000962F03C084918D9331969150D8F7F09397
:1002B0009D00E0939C007727C1CF962F02C08191CB
:1002C0008D939150E0F7F3CFCF91089584E690E0BD
:1002D00080939A000B968093990085B7836085BFC1
:1002E0008BB780648BBF08950F930FB70F93B09BAC
:1002F000FECFB09B06C0B09B04C0B09B02C0000004
:1003000000C01F933F932F9331E012E006B31027F4
:1003100010FD32E0102F3A95C9F700FDE4C006B396
:10032000102717952FE72795DF9316B30127079519
:100330002795CF93C0919A0006B31027179527955C
:100340003BE0DD274F9316B30127079527954FEF25
:10035000000055C0B09BFECFB09B06C0B09B04C050
:10036000B09B02C0000000C0DF9100C0CDCF16B32B
:10037000137079F1407C2C6F13C006B3037049F100
:1003800041782C6F15C0037021F1102F2C6F06B32C
:1003900019C006B30370E9F04E7F2C6F18C038F314
:1003A00006B30370B1F0102717952795243028F372
:1003B00016B3012707952795422749934FEF06B3B8
:1003C000243008F3102717952795243010F316B31F
:1003D0001370E1F10127079527952430F0F006B35B
:1003E0000370A1F11027179527952430E0F016B37C
:1003F0000127079527953A9541F12430D0F006B3AF
:10040000037021F11027179527952430C0F016B3FB
:100410000127079527952430C2CF16B31370B1F08A
:100420004C7F2C6FDCCF06B3037081F0487F2C6FBC
:10043000DECF16B3137051F0407F2C6FE0CF06B3C0
:10044000037021F0407E2C6FE2CF3AC03C2FC09168
:100450009A003C1B00E433300ABF90F108811981F7
:10046000412F1F77209198000D3271F1013E61F10B
:100470000936B9F0033C11F00B3411F510919F00CF
:100480001123F1F000919E000030B1F530939E00F1
:1004900010939B0000919900C093990000939A00DB
:1004A0002EC0121769F4309162003F3F29F10FEF1F
:1004B00000936200CDE8D0E025C0002700939F00A4
:1004C0004F91CF91DF910FC01217B9F700939F00A2
:1004D0000FEF00936300009362004F91CF910AB732
:1004E00006FD38CFDF9100E40ABF2F913F911F91A5
:1004F0000F910FBF0F911895C0E6D0E002C0C1E682
:10050000D0E032E05F9308B30C7F016008BB53E09A
:1005100017B3136017BB20E80FC0052710E008BB16
:1005200010C0052710E0089408BB13C0052710E091
:1005300015C0052710E019C020FF052708BB279527
:1005400017951C3F50F720FF0527279508BB1795E7
:100550001C3F38F720FF05272795179508BB1C3F40
:1005600028F720FF0527279517951C3F08BB08F79C
:1005700000C0499120FF052708BB279517951C3F10
:1005800048F520FF0527279508BB17951C3F30F538
:1005900020FF05272795179508BB1C3F20F520FF56
:1005A0000527279517951C3F08BB00F5242F3A9582
:1005B00019F60C7F5F9108BB34E03A95F1F70160C2
:1005C00017B31C7F08BB0C7F4F91CF9117BB08BBA3
:1005D000DF9189CF052710E008BBD1CF052710E0B8
:1005E000089408BBD4CF052710E0D6CF052710E02C
:1005F000DACFA82FB92F8FEF9FEF41E050EA61507B
:1006000070F02D9138E0722F782796958795269572
:1006100070FF02C0842795273A95A9F7F0CF8095FF
:100620009095089582E58DB981E08EB9089588236B
:1006300039F488E493E09093A1008093A00008959A
:1006400085E693E09093A1008093A000089592B76F
:1006500082B7891B8C30E0F3089587B38C6287BB27
:10066000C298C598F4DFC29AF2DFC2988091A000C8
:100670009091A1008556934009F00895D3DF089525
:1006800087B3837D87BB88B3837D88BB1DB80895FE
:100690000F931F93CF93C82F00E017E00CC0C398AF
:1006A000CC0F000FB4990F5FC59AD1DFC598CFDF8B
:1006B000115017FD04C0C7FFF2CFC39AF1CF802FAE
:1006C0009927CF911F910F9108958FB9779BFECFF6
:1006D0008FB1992708951F93CF93CFE103C0C150E5
:1006E000CF3F51F1E091A000F091A1008CEA099573
:1006F000E091A000F091A10083E50995E091A000B0
:10070000F091A10080E00995182FE091A000F091F0
:10071000A10080E00995133591F01DB8C59A97DFC7
:10072000C59895DF8091A0009091A10085569340D7
:10073000B1F678DFC150B0F681E090E002C080E011
:1007400090E0CF911F9108950F931F938C018170BA
:10075000880F880F880FE091A000F091A1008062BF
:100760000995C801892F99278695E091A000F091FD
:10077000A100099516950795E091A000F091A100C0
:10078000802F0995E091A000F091A10080E00995EB
:1007900099271F910F9108950F931F93CF93DF9384
:1007A000EC01062F142F8170880F880F880FE091BD
:1007B000A000F091A10080640995CE01892F9927AE
:1007C0008695E091A000F091A1000995CE01969543
:1007D0008795E091A000F091A1000995E091A0001B
:1007E000F091A100802F09951123A9F00F3789F00E
:1007F0001EE102B7CE01A8DF8F3769F482B7801BF4
:100800008D3310F002B711501123A1F781E090E071
:1008100004C08FE08CD080E090E0DF91CF911F91F9
:100820000F9108950F931F93CF93DF93EC01162F31
:10083000E091A000F091A1008CE40995CE01892FF0
:1008400099278695E091A000F091A1000995CE012D
:1008500096958795E091A000F091A1000995E0910F
:10086000A000F091A10080E009951F3F89F01EE1F2
:1008700002B7CE0169DF8F3F69F482B7801B8D33E9
:1008800010F002B711501123A1F781E090E004C0ED
:100890008FE04DD080E090E0DF91CF911F910F91DC
:1008A00008950F931F938C01E091A000F091A10097
:1008B00080EA0995812F9927E091A000F091A1008D
:1008C0000995E091A000F091A100802F0995E09199
:1008D000A000F091A10080E0099599271F910F9148
:1008E0000895FF920F931F938C01F62EE091A000C4
:1008F000F091A10080EC0995812F9927E091A0004B
:10090000F091A1000995E091A000F091A100802F45
:100910000995E091A000F091A1008F2D09958EE13D
:1009200006D080E090E01F910F91FF900895382F3E
:1009300020E0231740F492B782B7891B8C33E0F391
:100940002F5F2317C0F308951F93CF93DF93EC011C
:1009500010E089818130A1F0823009F472C08330C7
:1009600009F472C0843091F0873009F450C08530AA
:1009700009F4AAC0863039F1883009F0A9C086C0D0
:100980009A9B812F54DE69DEA998A2C08B8199279A
:10099000982F88272A813327822B932B90938900C5
:1009A000809388008F819927982F88272E8133275D
:1009B000822B932B90937E0080937D0082E0809326
:1009C0007F001FEF85C08B819927982F88272A8168
:1009D0003327822B932B90938900809388009C81EE
:1009E00090938A008D8180938B0080FF02C090934A
:1009F0008C008F819927982F88272E813327822B6F
:100A0000932B90937E0080937D0081E0D8CF8B81E3
:100A10009927982F88272A813327822B932B90930D
:100A20008900809388008F819927982F88272E81AD
:100A30003327822B932B90937E0080937D0083E05D
:100A4000BECF1EDEA99A44C0E091A000F091A100A3
:100A50008A81099580938000E091A000F091A10027
:100A60008B81099580938100E091A000F091A10015
:100A70008C81099580938200E091A000F091A10003
:100A80008D8109958093830014E022C08B81992782
:100A9000982F88272A813327822B932B90938900C4
:100AA0008093880010938A0010938B008F81992780
:100AB000982F88272E813327822B932B90937E00AB
:100AC00080937D0084E07BCF06DE8093800011E080
:100AD00080E890E090939D0080939C00812F99275F
:100AE000DF91CF911F910895EF92FF921F93CF93C3
:100AF0007C01162F90917F00892F8250823050F513
:100B0000C0E0C617C0F01FC0809188009091890096
:100B1000C8DEF701EC0FF11D808380918800909171
:100B2000890001969093890080938800CF5FC11758
:100B300050F490917F00923039F780918800909125
:100B4000890002DEE6CF183010F410927F00812F6A
:100B5000992702C08FEF90E0CF911F91FF90EF9007
:100B60000895CF92DF92EF92FF920F931F93CF934E
:100B7000DF936C01062F40917F00413019F0443023
:100B800009F073C010E01017F0F16CC080918A007A
:100B9000882309F046C0C12FDD27FE01EC0DFD1DA5
:100BA00060818091880090918900F6DD80917D00C0
:100BB00090917E00019790937E0080937D00892B19
:100BC000A1F410927F0080918B0081FF0EC0909164
:100BD0008C0080918A00981741F0CC0DDD1D688152
:100BE00080918800909189001DDE8091880090910D
:100BF0008900019690938900809388001F5F1017E9
:100C000088F540917F00413009F2C12FDD27FE01B8
:100C1000EC0DFD1D6081809188009091890061DE5E
:100C2000C5CFC12FDD277E01EC0CFD1C40E0F70194
:100C300060818091880090918900AEDD80918C0068
:100C4000815080938C00882309F0B0CFF701608138
:100C50008091880090918900E5DD80918A008093E1
:100C60008C00A4CF80E090E002C08FEF90E0DF9195
:100C7000CF911F910F91FF90EF90DF90CF9008954B
:100C8000CFE5D4E0DEBFCDBF12BA18BA8BEF81BB7F
:100C900017BA93E094BB8EEF85BB93BF81E0C7DCAE
:0A0CA00015DB789481DA80DAFDCFCD
:040CAA005AD2FFFF1C
:00000001FF
